:100000000C9452110C94FB110C94FB110C94FB11E9
:100010000C94FB110C94FB110C94FB110C94FB1130
:100020000C94FB110C94FB110C94FB110C94FB1120
:100030000C94FB110C9425130C94FB110C94FB11E4
:100040000C94FB110C94FB110C94FB110C94FB1100
:100050000C94FB110C94FB110C94FB110C94FB11F0
:100060000C94FB110C94FB110C94FB110C94FB11E0
:100070000000000000000000000000000000000080
:100080000000000000000000000000000000000070
:100090000000000000000000000000000000000060
:1000A0000000000000000000000000000000000050
:1000B0000000000000000000000000000000000040
:1000C0000000000000000000000000000000000030
:1000D00000000000000000400000000000494953FB
:1000E000000000404A52242D00004A491C2E2D1CBD
:1000F00000000000000000000000000000000040C0
:10010000000000004949525200494952521B1C1C30
:1001100049521B1C251C13091C2524130A0101012B
:1001200025130A0A0A0A0A0A0A0A0A0A0A0A0A0A0B
:100130000000000000000000494952525252525241
:100140005B1B12121309001C130A0A0A0A00132D62
:100150000101010A0001251B090A0A0000251C1CD7
:100160000A13010025251C1C130A0025252425251A
:1001700000000000000000004949490000000000A4
:100180001B13524949000000241C1C5B490000005D
:100190001C6D1C25524900001C1C652524490000CB
:1001A0001C1C652524490000241C6D2E1C490000E0
:1001B000000000000000000000000000000000013E
:1001C0000000000000005252000000000013522501
:1001D000000000000A522D25000000005B251300DE
:1001E0000000001B1300091C0000091B1C6D7F3759
:1001F0000052522E2E1C1313525C2E2513130A008C
:1002000025251C1C0A00000A25250A00000A2E3795
:100210001B0000132F37371C001B37372E2E2513DA
:1002200037372E2E2E2E1B1C2E2E2E37371C1C1C25
:100230000A0001130A0A0A13001213131313131CE2
:100240002E1C131313131C011C131313131C130064
:10025000131313131C1C001C1C1C1B1C2500123F19
:100260001C1C1C1D000A37251C1C1C130A2F2525CD
:100270001300132E252525250009372525252E2E8B
:10028000003725252E2E2513372E2E2E251C13251F
:10029000372E251C1C1C1C01251C1C1D1300001CBA
:1002A0001D1D0A00002E375B0100016E7F6E1213C8
:1002B00025256E1C5249000025251C135300000003
:1002C0001C1C1C524A0000001C13531B00000000A1
:1002D00001521C00000000005B1C00000000000038
:1002E0001B000000000000000000000000000000F3
:1002F0000000131B3F7F372E000013257F77777791
:100300000000136D7F77777700001B1BBF77BF76E8
:10031000000009136DBFBFBF0000001B125C77BF58
:10032000000000000A1B121B000000000000010A70
:10033000372E3777251C1C1C7776772D1C1C1C1C30
:1003400076772E1C1C1C1C2577761C1C24252D134F
:10035000BF65246D6E1B0001776D6D1B090A76BFAA
:100360001B5C1B121B645B121213131B120A090184
:100370001C1C1C252E1D010024252D24010009779D
:100380002D1B00000A7F7F7F000064BFBF7F1B1210
:1003900076BFBF6D1B121B096E1B12131B090000D9
:1003A000131209000000000000000000000000001F
:1003B00009777F7F131313007F7F1C0A1B00000047
:1003C00025121B0A000000001B09000000000000AD
:1003D000000000000000000000000000000000001D
:1003E000000000000000000000000000000000000D
:1003F00000000000000000000000000000000000FD
:1004000000000000000000000000000000000000EC
:10041000000000000000009B00000000009BE4AE14
:10042000000000529BA4777F00005B9B6D7F7F776D
:1004300000000000000000000000000000005BF66B
:100440000000005BFFFFFFFF00EDFFFFFFFFFFFF6E
:10045000EDF6FFFFFFFFFFB7BFBFBFFFFFFFFFB717
:100460007FBFBFFFFFFFFFBF6EB7BFFFFFFFFFBF35
:100470000000000000000000FFFFF6F6EDF6EDE4DE
:10048000FFFFB76E6D5C526EBFAE6D6565526577EE
:10049000AE655C5C52132E25AE6565524A37252544
:1004A000AE6E5B4A372E2525B76D5237372E2D2D70
:1004B0000000000000000000E49B9B4900000000D9
:1004C0002D65A49B520000006E2525A4520000005B
:1004D0002D6E252E5B00000025256E2D6D00000081
:1004E00025256E2E650000002525762F640000006E
:1004F0000000000000000000000000000000004AB2
:100500000000000000005B9B00000000005B9B2ED1
:10051000000000004A9B2E2E000000005B2E1C00F5
:100520000000005C1B000A250000095B1C6E7F7F39
:10053000405B5B777F6E656E5B65372E2525655B5F
:100540002D2E25251C4A526D2E2D1309095C7FBFC7
:100550001C00011C7F7FBFBF001C3F7F7F7F7FB7D8
:10056000373F77777F7F77BF3737777F7F6E77BF6C
:100570006EA4B7FFFFFFFFBFA4BFFFFFFFFFFFBFDA
:10058000BFBFFFFFFFFFFFAEBFBFFFFFFFFFBFA467
:10059000BFBFFFFFFFFFADBFBFFFFFFFFFF6FFFFC6
:1005A000BFFFFFFFFFFFFFBFBFFFFFFFFFFFBFBF9B
:1005B000B75B6D3F2E2E2E2EA4647F772E2E2E2E0F
:1005C000A47F7F7737372E1CBF7F7F7F2E251C258A
:1005D000BFBF7F2E25251C09BF776E2E1C09012564
:1005E0007F771B090A6E7F646452527FBF775B5C22
:1005F0002E2E76255B0000002D2D1C1B5B000000BD
:100600002524255B520000001C1C5B5C00000000E0
:100610000A5B640000000000646400000000000049
:100620005C0000000000000000000000000000006E
:1006300000001B5C7FBF773700001C6D7FBF7777A2
:1006400000001C6E7FBF7F7F00001C64BFBFBFBF68
:1006500000000A5C76BFBFFF00000065646DBFFF4D
:10066000000000005B6D646D0000000000000A1BCC
:1006700077777F7F376E7FBF777F7F776E777FBF9C
:100680007FBF7F2D76777FBFBF7F2D6E777FBFBF08
:10069000FF7776BFBF76A4AEBFBFBF7664AEFFFF65
:1006A000ADB6B6AEBFFFFFFF646DADB6AD645B0A1D
:1006B000BFFFFFFFFFBFAE5BBFFFFFFFF6ADAEFFAB
:1006C000BFFFFFFFFFFFFFFFADF6FFFFFFFFFFB61E
:1006D000FFFFFFFFFFFFBF5BFFFFFFFFFF5C0000AF
:1006E000FFFFA40000000000000000000000000068
:1006F00064BFBFBF64645C00FFBF765C6D0900002F
:10070000BF656D5B00000000765300000000000034
:1007100000000000000000000000000000000000D9
:1007200000000000000000000000000000000000C9
:10073000000000000000000000002600000026006D
:1007400000002F0000002F000000370000003700DD
:100750000000FF000000FF000000BF000000BF001D
:1007600000003700003700000000002626000000CF
:10077000000000000000000026262626260026266F
:10078000000000002F002F0000000037000037009D
:100790000000FF000000FFFF00BF00000000BF00DE
:1007A00037000000000037002626262626002626D1
:1007B000000000000000000026262600262626262F
:1007C000000000002F0000000000000037000000C3
:1007D000FFFF0000FFFFFFFF00000000BF00000060
:1007E00000000000370000002626260026262626C8
:1007F0000000000000000000000000002626260087
:100800002F00002F00002F003700370000003700B6
:100810000000FF000000FF00BF00BF000000BF009D
:1008200037003700003700000000262626000000B1
:10083000000000000000000026000000260000006C
:100840002F0000002F0000000037003700000000DC
:100850000000FF000000000000BF00BF000000001B
:1008600037000000370000002600000026000000CE
:100870000503000102030405060708090A0B0C0D15
:10088000000503000E0F1011121314151617181976
:100890001A0005011B1C1D1E1F000208000855043C
:1008A000085A0000F8000990000A1E32050000FFF7
:1008B00000000099080000000015232323AD2387C2
:1008C000277127262335234423572752236023FFEC
:1008D000FFFFFFFFFFFFFFFFFFFFFFFFFFFFFFFF28
:1008E000FFFFFFFFFFFFFFFFFFFFFFFFFFFFFFFF18
:1008F000FFFFFFFFFFFFFFFFFFFFFFFFFFFFFFFF08
:10090000FFFFFFFFFFFFFFFFFFFFFFFFFFFFFF00F6
:1009100000000000000000000000000000000000D7
:1009200000000000000000000000000000000000C7
:1009300000000000000000000000000000000000B7
:1009400000000000000000000000000000000000A7
:100950000000000000FFFF000000000000FFFF009B
:100960000000000000000000000000000000000087
:100970000000000000000000000000000000000077
:100980000000000000FFFF000000000000FFFFFF6C
:10099000FF000000000000FFFF000000000000005A
:1009A0000000000000000000000000000000000047
:1009B000000000000000000000000000000000FF38
:1009C000FF000000000000FFFF000000000000FF2B
:1009D000FFFFFFFFFFFFFF0000000000000000001E
:1009E000000000000000000000000000000000FF08
:1009F000FFFFFFFFFFFFFF000000000000000000FE
:100A000000000000000000000000000000000000E6
:100A100000000000000000000000000000000000D6
:100A200000000000000000000000000000000000C6
:100A300000000000000000000000000000000000B6
:100A400000000000000000000000000000000000A6
:100A500000FBFBFB0000000000FBFBFB00000000B4
:100A600000B8B8B80000000000707000000000007E
:100A70000070700000000000000000000000000096
:100A80000020200000000000000000000000000026
:100A900000FB00FB0000000000FB00FB000000006A
:100AA00000B800B8000000000000000000000000D6
:100AB0000000000000000000000000000000000036
:100AC0000000000000000000000000000000000026
:100AD000FB000000FB0000FBFBFBFBFBFBFB000043
:100AE000B8000000B80000007000000070000000B6
:100AF0007000000070000020202020202020000036
:100B000020000000200000000000000000000000A5
:100B10000000FB0000000000FBFBFBFBFBFB00B840
:100B20000000B800000000007070707070000000DD
:100B30000000700000700020202020202000000015
:100B4000000020000000000000000000000000FB8A
:100B5000FB000000000000FBFB0000FB00000000A9
:100B60000000B8000000000000700000000000005D
:100B700070000000000000200000202000000000A5
:100B80000000202000000000000000000000000025
:100B900000FBFB0000000000FB0000FB0000000069
:100BA000B8B800B80000000070707000000000705D
:100BB0000000707000700020000000202000000085
:100BC0002020202000200000000000000000000085
:100BD000FBFB000000000000FBFB00000000000029
:100BE00000B80000000000007000000000000000DD
:100BF00000000000000000000000000000000000F5
:100C000000000000000000000000000000000000E4
:100C1000000000FBFB0000000000FB0000000000E3
:100C200000B800000000000000700000000000009C
:100C30000070000000000000000020000000000024
:100C40000000002020000000000000000000000064
:100C500000FBFB0000000000000000FB00000000A3
:100C600000000000B800000000000000700000005C
:100C700000000000700000000000002000000000E4
:100C80000020200000000000000000000000000024
:100C900000000000000000000000FB000000000059
:100CA000B800B800B80000000070707000000000CC
:100CB00070007000700000000000200000000000C4
:100CC0000000000000000000000000000000000024
:100CD00000000000000000000000FB000000000019
:100CE0000000B8000000000070707070700000001C
:100CF0000000700000000000000020000000000064
:100D000000000000000000000000000000000000E3
:100D100000000000000000000000000000000000D3
:100D200000000000000000000000000000000000C3
:100D30000070700000000000002020000000000093
:100D40002020000000000000000000000000000063
:100D50000000000000000000000000000000000093
:100D60000000000000000000707070707000000053
:100D70000000000000000000000000000000000073
:100D80000000000000000000000000000000000063
:100D90000000000000000000000000000000000053
:100DA0000000000000000000000000000000000043
:100DB00000000000000000000020200000000000F3
:100DC00000202000000000000000000000000000E3
:100DD0000000000000FB000000000000FB0000001D
:100DE000000000B8000000000000700000000000DB
:100DF0000070000000000000200000000000002043
:100E000000000000000000000000000000000000E2
:100E100000FFFFFF00000000FF0000FFFF0000AD2B
:100E2000AD000000ADAD00ADAD000000ADAD005BAC
:100E30005B0000005B5B00005B5B00005B00000090
:100E4000005B5B5B00000000000000000000000091
:100E50000000FFFF0000000000FFFFFF0000000097
:100E60000000ADAD000000000000ADAD00000000CE
:100E700000005B5B0000000000005B5B0000000006
:100E80005B5B5B5B5B5B0000000000000000000040
:100E9000FFFFFFFFFF0000FFFF000000FFFF00005B
:100EA000000000FFFFFF000000ADADADAD00000091
:100EB000ADADADAD0000005B5B5B00000000005B12
:100EC0005B5B5B5B5B5B0000000000000000000000
:100ED000FFFFFFFFFFFF0000000000FFFF0000001A
:100EE0000000ADAD0000000000ADADADAD000000F4
:100EF000000000005B5B005B5B0000005B5B0000D0
:100F00005B5B5B5B5B00000000000000000000001A
:100F10000000FFFFFF00000000FFFFFFFF000000D8
:100F2000ADAD00ADAD0000ADAD0000ADAD00005BFE
:100F30005B5B5B5B5B5B00000000005B5B000000D9
:100F40000000005B5B00000000000000000000FFEC
:100F5000FFFFFFFFFF0000FFFF000000000000ADEB
:100F6000ADADADADAD00000000000000ADAD0000C6
:100F7000000000005B5B005B5B0000005B5B00004F
:100F80005B5B5B5B5B00000000000000000000009A
:100F900000FFFFFFFF000000FFFF0000000000ADAA
:100FA000AD000000000000ADADADADADAD00005B2B
:100FB0005B0000005B5B005B5B0000005B5B0000B4
:100FC0005B5B5B5B5B00000000000000000000FF5B
:100FD000FFFFFFFFFFFF00FFFF000000FFFF00001B
:100FE000000000ADAD0000000000ADAD000000004D
:100FF000005B5B0000000000005B5B000000000085
:10100000005B5B000000000000000000000000002A
:10101000FFFFFFFF000000FFFF000000FF0000AD2A
:10102000ADAD0000AD000000ADADADAD0000005BAA
:1010300000005B5B5B5B005B000000005B5B000033
:101040005B5B5B5B5B0000000000000000000000D9
:10105000FFFFFFFFFF0000FFFF000000FFFF00ADEC
:10106000AD000000ADAD0000ADADADADADAD00006B
:10107000000000005B5B00000000005B5B00000004
:101080005B5B5B5B000000000000000000000000F4
:10109000000000000000000000FBFB00000000005A
:1010A00000B8B800000000000000000000000000D0
:1010B0000070700000000000002020000000000010
:1010C0000000000000000000000000000000000020
:1010D000000000000000000000FBFB00000000001A
:1010E00000B8B80000000000000000000000000090
:1010F00000707000000000000020200000000000D0
:10110000202000000000000000000000000000009F
:10111000000000FB000000000000FB0000000000D9
:1011200000B8000000000000700000000000000097
:10113000007000000000000000002000000000001F
:10114000000000200000000000000000000000007F
:10115000000000000000000000000000000000008F
:10116000B8B8B8B8B80000000000000000000000E7
:10117000707070707000000000000000000000003F
:10118000000000000000000000000000000000005F
:1011900000FB0000000000000000FB000000000059
:1011A000000000B800000000000000007000000017
:1011B000000000700000000000002000000000009F
:1011C00000200000000000000000000000000000FF
:1011D000FBFBFBFBFB0000FBFBFBFBFBFBFB00B893
:1011E000B8000000B8B800000000007070000000F7
:1011F000007070700000000000000000000000009F
:10120000002020200000000000000000000000007E
:1012100000FBFBFB00000000FB000000FB0000B82F
:101220000000B800B800007000700070700000701E
:1012300000007070000000002000000000000000AE
:10124000002020202000000000000000000000001E
:1012500000FBFBFB00000000FBFB00FBFB0000B8F9
:10126000B8000000B8B80070700000007070007026
:10127000707070707070002020000000202000202E
:10128000200000002020000000000000000000FB03
:10129000FBFBFBFBFB0000FBFB000000FBFB00B8C3
:1012A000B8000000B8B80070707070707000007006
:1012B000700000007070002020000000202000203E
:1012C000202020202000000000000000000000007E
:1012D00000FBFBFBFB000000FBFB0000FBFB00B87E
:1012E000B8000000000000707000000000000070F6
:1012F00070000000000000002020000020200000FE
:10130000002020202000000000000000000000FB62
:10131000FBFBFBFB000000FBFB0000FBFB0000B83D
:10132000B8000000B8B80070700000007070007065
:1013300070000000707000202000002020000020BD
:10134000202020200000000000000000000000FB22
:10135000FBFBFBFBFBFB00FBFB000000000000B8FD
:10136000B8000000000000707070707070000070B5
:10137000700000000000002020000000000000209D
:10138000202020202020000000000000000000FBA2
:10139000FBFBFBFBFBFB00FBFB000000000000B8BD
:1013A000B800000000000070707070707000007075
:1013B000700000000000002020000000000000205D
:1013C00020000000000000000000000000000000FD
:1013D00000FBFBFBFBFB0000FBFB0000000000B878
:1013E000B8000000000000707000007070700070A5
:1013F000700000007070000020200000202000001D
:10140000002020202020000000000000000000FB41
:10141000FB000000FBFB00FBFB000000FBFB00B837
:10142000B8000000B8B80070707070707070007014
:1014300070000000707000202000000020200020BC
:10144000200000002020000000000000000000003C
:10145000FBFBFBFBFBFB00000000FBFB00000000B4
:101460000000B8B80000000000007070000000002C
:10147000000070700000000000002020000000004C
:10148000202020202020000000000000000000009C
:101490000000FBFBFBFB0000000000FBFB0000006A
:1014A000000000B8B80000000000007070000000EC
:1014B00000000070700000200000002020000000EC
:1014C000202020200000000000000000000000FBA1
:1014D000FB000000FBFB00FBFB0000FBFB0000B877
:1014E000B800B8B8000000707070700000000070A4
:1014F000707070700000002020002020200000206C
:10150000200000202020000000000000000000005B
:10151000FBFB000000000000FBFB000000000000DF
:10152000B8B800000000000070700000000000006B
:10153000707000000000000020200000000000008B
:10154000202020202020000000000000000000FBE0
:10155000FB000000FBFB00FBFBFB00FBFBFB00B800
:10156000B8B8B8B8B8B800707070707070700070AB
:10157000700070007070002020000000202000200B
:10158000200000002020000000000000000000FB00
:10159000FB000000FBFB00FBFBFB0000FBFB00B8BB
:1015A000B8B8B800B8B80070707070707070007023
:1015B000700070707070002020000020202000203B
:1015C00020000000202000000000000000000000BB
:1015D000FBFBFBFBFB0000FBFB000000FBFB00B880
:1015E000B8000000B8B800707000000070700070A3
:1015F000700000007070002020000000202000001B
:10160000202020202000000000000000000000FB3F
:10161000FBFBFBFBFB0000FBFB000000FBFB00B83F
:10162000B8000000B8B80070700000007070007062
:10163000707070707000002020000000000000201A
:10164000200000000000000000000000000000007A
:10165000FBFBFBFBFB0000FBFB000000FBFB00B8FF
:10166000B8000000B8B80070700000007070007022
:1016700070007070707000202000002020000000BA
:10168000202020200020000000000000000000FBBF
:10169000FBFBFBFBFB0000FBFB000000FBFB00B8BF
:1016A000B8000000B8B80070700000707070007072
:1016B00070707070000000202000202020000020AA
:1016C000200000202020000000000000000000009A
:1016D000FBFBFBFB000000FBFB0000FBFB0000B87A
:1016E000B800000000000000707070707000000012
:1016F000000000007070002020000000202000008A
:101700002020202020000000000000000000000039
:10171000FBFBFBFBFBFB00000000FBFB00000000F1
:101720000000B8B800000000000070700000000069
:101730000000707000000000000020200000000089
:10174000000020200000000000000000000000FB5E
:10175000FB000000FBFB00FBFB000000FBFB00B8F4
:10176000B8000000B8B80070700000007070007021
:101770007000000070700020200000002020000099
:10178000202020202000000000000000000000FBBE
:10179000FB000000FBFB00FBFB000000FBFB00B8B4
:1017A000B8000000B8B80070707000707070000071
:1017B0007070707070000000002020200000000099
:1017C000000020000000000000000000000000FBFE
:1017D000FB000000FBFB00FBFB000000FBFB00B874
:1017E000B800B800B8B80070707070707070007099
:1017F0007070707070700020202000202020002069
:10180000200000002020000000000000000000FB7D
:10181000FB000000FBFB00FBFBFB00FBFBFB0000F5
:10182000B8B8B8B8B80000000070707000000000D0
:101830007070707070000020202000202020002098
:101840002000000020200000000000000000000038
:10185000FBFB0000FBFB0000FBFB0000FBFB0000B0
:10186000B8B80000B8B800000070707070000000D8
:101870000000707000000000000020200000000048
:10188000000020200000000000000000000000FB1D
:10189000FBFBFBFBFBFB0000000000FBFBFB000075
:1018A0000000B8B8B80000000070707000000000C0
:1018B0007070700000000020202000000000002058
:1018C0002020202020200000000000000000000058
:1018D00000FBFBFBFB00000000FBFB000000000026
:1018E00000B8B800000000000070700000000000A8
:1018F00000707000000000000020200000000000C8
:101900000020202020000000000000000000000057
:1019100000FFFFFFFF000000FF00000000FF00FFCE
:101920000000FFFF0000FFFF00FF00000000FFFFBE
:1019300000FF00000000FFFF0000FFFF0000FF00AD
:10194000FF00000000FF000000FFFFFFFF0000009D
:1019500000FBFBFBFB000000000000FBFB000000A5
:10196000000000B8B8000000000000707000000027
:101970000000007070000000000000202000000047
:1019800000202020200000000000000000000000D7
:1019900000FB000000000000B800B800000000706C
:1019A00000000070000000000000000000000000C7
:1019B0000000000000000000000000000000000027
:1019C0000000000000000000000000000000000017
:1019D0000000000000000000000000000000000007
:1019E00000000000000000000000000000000000F7
:1019F00000000000000000000000000000000020C7
:101A00002020202020200000000000000000001EF8
:101A1000001C0000000000000000000000000000AA
:101A200000000000000000000000000000000000B6
:101A300000000000000000000000000000000000A6
:101A40000000000000000000000000000000000195
:101A5000000100010001000100010001000100017E
:101A6000000100010001000100010002000300016B
:101A7000000100010001000100010001000100015E
:101A8000000100010001000100010001000100014E
:101A9000000100010001000100010001000100013E
:101AA000000100010001000200030001000100012B
:101AB000000100010001000100010001000100011E
:101AC000000100010001000100010001000100010E
:101AD00000010001000100010001000100010001FE
:101AE00000010002000300010001000100010001EB
:101AF00000010001000100010001000100010001DE
:101B000000010001000100010001000100010001CD
:101B100000010001000100010001000100010002BC
:101B200000030001000100010001000100010001AB
:101B3000000100010001000100010001000100019D
:101B4000000100010001000100010001000100018D
:101B5000000100010001000100010002000300017A
:101B6000000100010001000100010001000100016D
:101B7000000100010001000100010001000100015D
:101B8000000100010001000100010001000100014D
:101B9000000100010001000200030001000100013A
:101BA000000100010001000100010001000100012D
:101BB000000100010001000100010001000100011D
:101BC000000100010001000100010001000100010D
:101BD00000010002000300010001000100010001FA
:101BE00000010001000100010001000100010001ED
:101BF00000010001000100010001000100010001DD
:101C000000010001000100010001000100010002CB
:101C100000030001000100010001000100010001BA
:101C200000010001000100010001000100010001AC
:101C3000000100010001000100010001000100019C
:101C40000001000100010001000100020003000189
:101C5000000100010001000100010001000100017C
:101C6000000100010001000100010001000100016C
:101C7000000100010001000100010001000100015C
:101C80000001000100010002000300010001000149
:101C9000000100010001000100010001000100013C
:101CA000000100010001000100010001000100012C
:101CB000000100010001000100010001000100011C
:101CC0000001000200030001000100010001000109
:101CD00000010001000100010001000100010001FC
:101CE00000010001000100010001000100010001EC
:101CF00000010001000100010001000100010002DB
:101D000000030001000100010001000100010001C9
:101D100000010001000100010001000100010001BB
:101D200000010001000100010001000100010001AB
:101D30000001000100010001000100020003000198
:101D4000000100010001000100010001000100018B
:101D5000000100010001000100010001000100017B
:101D6000000100010001000100010001000100016B
:101D70000001000100010002000300010001000158
:101D8000000100010001000100010001000100014B
:101D9000000100010001000100010001000100013B
:101DA000000100010001000100010001000100012B
:101DB0000001000200030001000100010001000118
:101DC000000100010001000100010001000100010B
:101DD00000010001000100010001000100010001FB
:101DE00000010001000100010001000100010002EA
:101DF00000030001000100010001000100010001D9
:101E000000010001000100010001000100010001CA
:101E100000010001000100010001000100010001BA
:101E200000010001000100010001000200030001A7
:101E3000000100010001000100010001000100019A
:101E4000000100010001000100010001000100018A
:101E5000000100010001000100010001000100017A
:101E60000001000100010002000300010001000167
:101E7000000100010001000100010001000100015A
:101E8000000100010001000100010001000100014A
:101E9000000100010001000100010001000100013A
:101EA0000001000200030001000100010001000127
:101EB000000100010001000100010001000100011A
:101EC000000100010001000100010001000100010A
:101ED00000010001000100010001000100010002F9
:101EE00000030001000100010001000100010001E8
:101EF00000010001000100010001000100010001DA
:101F000000010001000100010001000100010001C9
:101F100000010001000100010001000200030001B6
:101F200000010001000100010001000100010001A9
:101F30000001000100010001000100010001000199
:101F40000001000100010001000100010001000189
:101F50000001000100010002000300010001000176
:101F60000001000100010001000100010001000169
:101F70000001000100010001000100010001000159
:101F80000001000100010001000100010001000149
:101F90000001000200030001000100010001000136
:101FA0000001000100010001000100010001000129
:101FB0000001000100010001000100010001000119
:101FC0000001000100010001000100010001000208
:101FD00000030001000100010001000100010001F7
:101FE00000010001000100010001000100010001E9
:101FF00000010001000100010001000100010001D9
:1020000000010001000100010001000200030001C5
:1020100000010001000100010001000100010001B8
:1020200000010001000100010001000100010001A8
:102030000001000100010001000100010001000198
:102040000001000100010002000300010001000185
:102050000001000100010001000100010001000178
:10206000000100010001000000000000000000006D
:102070000000000000000000000000000000000060
:102080000000000000000000000000000000000050
:102090000000000000000000000000000000000040
:1020A000000000010400000000040005000400041A
:1020B0000004000400040001000100040004000109
:1020C00000010004000400010001000400040004F9
:1020D00000040004000400050001000100010004E8
:1020E00000010001000100040001000100010004E2
:1020F00000010001000100040001000100010004D2
:1021000000040005000400040004000400010001B4
:1021100000010004000400040004000400040001A5
:102120000001000100040004000400040004000594
:102130000004000400040004000100010001000488
:10214000000100040004000400010001000100047B
:102150000004000400040004000400050004000161
:10216000000100010004000100010004000400045B
:10217000000400040001000100010004000100014E
:102180000001000400040005000400040004000431
:102190000004000100010001000400040004000428
:1021A0000001000100010004000400040004000418
:1021B0000004000500040004000400010004000104
:1021C00000010001000400040004000400040001F8
:1021D00000010004000400040004000400040005E1
:1021E00000040004000400040001000100010004D8
:1021F00000010001000100040001000100010004D1
:1022000000010001000100040004000500040004B6
:1022100000040004000400010001000400040004A4
:102220000004000400040001000100040004000494
:10223000000400040004000500040004000400047D
:102240000004000100010004000400040004000474
:10225000000100010001000400010004000400046A
:10226000000007FF0003500008CE03070000FF0036
:1022700007FF00041402070000FF0007FF000332FD
:102280000008CE0D070000FF0000006122000000E2
:10229000000000006F22000000000000007A220011
:1022A0000000000011241FBECFEFD0E1DEBFCDBF84
:1022B00014BE88E10FB6F89480936000109260001D
:1022C0000FBE12E0A0E0B1E0EAEAF8E502C0059036
:1022D0000D92A433B107D9F71FE0A4E3B2E001C027
:1022E0001D92A534B107E1F7F894E1E6FCE080E047
:1022F00090E020E802C02193019632E08C309307F1
:10230000D4F381E69CE090936E0E80936D0E109254
:102310006F0EE2E7FEE080E090E003C010820196DD
:102320003A9684309105D4F381E08093920E8093A5
:10233000930E8093910E1092810015BCE4E1FFE0B2
:1023400080E090E020EE03C02083019634968A302E
:102350009105D4F39093A70E8093A60E8FEF87B9C3
:1023600084B980E88AB98CE081B98BEF82B9109288
:10237000330C86E08093340C109285001092840018
:1023800083E0809389008DE88093880089E08093C2
:10239000810082E080936F0082E484BD17BC91E0ED
:1023A00095BD83E88093B0001092B3009093B10084
:1023B00081E185B91092440C1092370C1092380CC0
:1023C00010923F0C10923E0C1092430C1092420C53
:1023D0001092A80E0E94272280E00E94131580FF11
:1023E00003C084E00E94101578940E94B0220E94DD
:1023F000DC2B0C94532C0C94000064136E137C1390
:10240000D012E6EEFBE0C0E4D2E020913D0F0027C1
:10241000A081B181AC0FBD1F1C911283021708F47B
:10242000102F1C9333960395093190F309E4095159
:1024300016E01A95F1F70A95D9F716E01A95F1F713
:1024400000C0C0E4D2E000EEA02E662778E02DD1D7
:1024500033E23A95F1F70E9467123FE03A95F1F7BF
:1024600000C0AA94A9F00000639500000000683045
:1024700029F0C895C895C8950000E9CF66270024C3
:102480003EE1C30FD01D0000000000000000DFCFC0
:10249000C895C895C895C895C8950000000005D195
:1024A0000E949C2711E00091360C01270093360C06
:1024B0002091370C002309F021272093370CE1E00D
:1024C000E093350CE2E0E093360011240895DE013C
:1024D000679F00000091390C10913A0C005416408F
:1024E000000D111D180106EA15E0000D111D28014F
:1024F00030E41EE12D9129316FB660FA239FA101CE
:102500000EF4A201040E151EF001F6F0059108B9B3
:102510002D91059108B9239F059108B929316FB60E
:10252000059108B908F4A201059108B960FA040EF2
:10253000059108B9151E1A95059108B9059139F14B
:10254000F00108B91EF700C0019108B92D91019161
:10255000000008B9239F0191000008B929316FB626
:1025600060FA019108B90EF0A1010191040E08B9B9
:10257000151E00C0019108B9000000C0019108B902
:1025800001911A9521F0F00108B906F6DDCF08B9DE
:102590000027C895000008B905E00A95F1F70895ED
:1025A00028980E94A216E7E1EA95F1F7289AE3D06D
:1025B000E0E0F6E0C6D0E0FF05D0E0FF02C00E94F8
:1025C000C7150895EF93E091340CE93EE0F5E9304A
:1025D000D0F12F923F924F925F926F927F928F92A3
:1025E0009F92AF92BF92CF92DF92EF92FF920F93A2
:1025F0001F932F933F934F935F936F937F938F938B
:102600009F93AF93BF93CF93DF930E940112DF910B
:10261000CF91BF91AF919F918F917F916F915F917A
:102620004F913F912F911F910F91FF90EF90DF906D
:10263000CF90BF90AF909F908F907F906F905F9062
:102640004F903F902F90EF910895FF93EF93EFB746
:10265000EF93E0918400EE50E13000F0E23000F0C2
:10266000E33000F0E43000F0E53000F0E63000F058
:10267000E73000F0E83000F0E93000F005D0EF91ED
:10268000EFBFEF91FF9118950F921F92EAEFF3E2DF
:102690000090330C000C1124E00DF11D05901490F6
:1026A000F00109951F900F90089528980E94A21696
:1026B000E5E1EA95F1F7E091340CEA95E093340C0A
:1026C000289A00000000089528980E94CB16289AA6
:1026D0000000E1E0F6E035D047D0089528980E9448
:1026E000CB16E0EB0000EA95E9F700000000289A1D
:1026F000F6E0E2E026D0089528980E94CB16289AAA
:102700000000E3E0FDEF1DD0E091340CE53091F4E2
:10271000E091360CE1300000F091440C19F4F09196
:10272000440CF195E3E0E0938900EDE8EF0FE093CE
:1027300088000895E3E0E0938900EDE8E0938800E5
:1027400008950090340C0A9410905F0011FC0F2E35
:102750000092340C0090330C11FC0E2E0092330CBE
:10276000E0E011FCE1E00895E3E0E0938900EDE8AA
:10277000E09388000895E7E0E0938900EBE1E093BF
:1027800088000895E6E6F3E0A0E4B2E069E16D9325
:102790003197E9F711240895CC03CC03CC03CC0383
:1027A000CC03CC03CC03CC03CC03CC03CC03CC03B1
:1027B000CC03CC03CC03CC03CC03CC03CC03CC03A1
:1027C000CC03CC03CC03CC03CC03CC03CC03CC0391
:1027D000CC03CC03CC03CC03CC03CC03CC03CC0381
:1027E000CC03CC03CC03CC03CC03CC03CC03CC0371
:1027F000CC03CC03CC03CC03CC03CC0399277727A1
:102800002EE1629F080E191EA0E4B2E0A00DB11DDA
:10281000475E4C9311240895089599272EE1629FF5
:10282000080E191EA0E4B2E0A00DB11D50913B0CA2
:10283000450F4C931124089580933B0C0895809389
:10284000310C9093320C08958093390C90933A0C8C
:1028500008958091350C089511241092350C089537
:1028600080E891E08093610090936100089580E892
:1028700090E08093610090936100089520E4E091DE
:10288000390CF0913A0C8951829FE00DF11DA6EAB6
:10289000B5E0629FA00DB11D002405900D9205903A
:1028A0000D9205900D9205900D9205900D92059058
:1028B0000D9205900D9205900D9205900D92059048
:1028C0000D9205900D9205900D9205900D92059038
:1028D0000D9205900D9205900D9205900D92059028
:1028E0000D9205900D9205900D9205900D92059018
:1028F0000D9205900D9205900D9205900D92059008
:102900000D9205900D9205900D9205900D920590F7
:102910000D9205900D9205900D9205900D920590E7
:102920000D9205900D9205900D9205900D920590D7
:102930000D9205900D9205900D9205900D920590C7
:102940000D9205900D9205900D9205900D920590B7
:102950000D9205900D9205900D9205900D920590A7
:102960000D9205900D9205900D9205900D92059097
:102970000D9205900D9205900D9205900D92059087
:102980000D9205900D9205900D9205900D92059077
:102990000D9205900D9205900D921124089594E0EA
:1029A000899FE3E1FFE0E00DF11D8281E091310CB0
:1029B000F091320C90E4899FE00DF11DA6EAB5E09C
:1029C000699FA00DB11D1124403021F4A20FB11D4B
:1029D000822F04C088E0821BE80FF11D503031F4D3
:1029E00098E0939FA00DB11D932F06C098E0931B14
:1029F00058E0599FE00DF11D11243EEF58E0591B9E
:102A000048E0481B259123132C9311964A95D1F742
:102A1000E80FF11DA80FB11D5A9591F711240895E3
:102A20008093440C0895882329F480913C0C909164
:102A30003D0C08958091400C9091410C089588239D
:102A400029F480913E0C90913F0C08958091420CA6
:102A50009091430C089578E07A95F1F70000019782
:102A6000D1F70895F999FECF92BD81BD60BDF8946C
:102A7000FA9AF99A78940895F999FECF92BD81BD9A
:102A8000F894F89A80B5789408950000000000004A
:102A90000000000000000000000000000000000036
:102AA0000000000000000000000000000000000026
:102AB0000000000000000000000000000000000016
:102AC0000000000000000000000000000000000006
:102AD00000000000000000000000000000000000F6
:102AE00000000000000000000000000000000000E6
:102AF00000000000000000000000000000000000D6
:102B000099277727833008F00895E0E0F8E3660F0F
:102B1000771FE60FF71FA591B491E2E7FEE02AE0E8
:102B2000289FE00DF11DA183B28311240895909197
:102B3000910E9170880F892B8093910E089599279B
:102B40007727E2E7FEE02AE0289FE00DF11D6E3FC7
:102B500031F46091910E6E7F6093910E0BC06F3FC8
:102B600031F46091910E6E6F6093910E03C07EE21E
:102B7000760F75831124089599277727E2E7FEE001
:102B80002AE0289FE00DF11D6083112408952F9302
:102B90003F934F935F936F937F938F939F93AF93E5
:102BA000BF93789411240E942C280E94B4280E947C
:102BB00070220E9481242F923F924F925F926F92D7
:102BC0007F928F929F92AF92BF92CF92DF92EF92BD
:102BD000FF920F931F93CF93DF9300906F0E00200F
:102BE00019F4A1E6BCE002C0A7E6BDE001E00026C2
:102BF00000926F0E02E00093700E5091900E609163
:102C0000920E7091930E8091940E2090730E3090DE
:102C1000740E4090760E5090770E6090750E109165
:102C2000720E70907D0E80907E0E90907F0EA09020
:102C3000800EB090810E20917C0EC090870ED090B7
:102C4000880EE0908A0EF0908B0E0091890E3091E4
:102C5000860E9FEF620C431CF20144914103002455
:102C60000008C12DD02D970CA81CF50144914203FA
:102C700000240008C10DD01D0C0DED1CF70144917E
:102C8000430300240008C10DD01D8A956AF44091C9
:102C9000910E842F8695062E0694062600FA7695C8
:102CA000679576F940FF66F940E860FD4FE7450318
:102CB00000240008C10DD01D0024C038D0050CF040
:102CC000CFE70A94C038D0050CF4C0E8C058CD93C3
:102CD0009A9509F0BFCF4091700E4A954093700EBF
:102CE00097E009F0B7CF6092750E4092760E909201
:102CF0007F0EA092800E0093890EE0928A0E609360
:102D0000920E7093930E8093940EDF91CF911F914A
:102D10000F91FF90EF90DF90CF90BF90AF909F907A
:102D20008F907F906F905F904F903F902F90BF91CA
:102D3000AF919F918F917F916F915F914F913F9153
:102D40002F9108950C94A4160C94A6160F931F931C
:102D50002ABDE0916D0EF0916E0E0191000000937E
:102D6000B3000EE0ED36F00710F40000000010F0A4
:102D7000E1E6FCE0E0936D0EF0936E0EC895C89509
:102D8000C895C895C895C8950000000000002AB5F0
:102D90001F910F9108950000E091340CE0FFD6CF11
:102DA000E1E1EA95F1F7000000000895000000005D
:102DB0000000000000000000000000000000000013
:102DC0000000000000000000000000000000000003
:102DD00000000000000000000000000000000000F3
:102DE00000000000000000000000000000000000E3
:102DF00000000000000000000000000000000000D3
:102E0000000306090C101316191C1F2225282B2E4F
:102E1000313336393C3F414447494C4E5153555864
:102E20005A5C5E60626466686A6B6D6F7071737421
:102E3000757678797A7A7B7C7D7D7E7E7E7F7F7FDA
:102E40007F7F7F7F7E7E7E7D7D7C7B7A7A797876C0
:102E500075747371706F6D6B6A68666462605E5CD6
:102E60005A585553514E4C494744413F3C393633EB
:102E7000312E2B2825221F1C191613100C090603AE
:102E800000FDFAF7F4F0EDEAE7E4E1DEDBD8D5D2B5
:102E9000CFCDCAC7C4C1BFBCB9B7B4B2AFADABA880
:102EA000A6A4A2A09E9C9A9896959391908F8D8CA3
:102EB0008B8A8887868685848383828282818181CA
:102EC0008181818182828283838485868687888AC4
:102ED0008B8C8D8F9091939596989A9C9EA0A2A48E
:102EE000A6A8ABADAFB2B4B7B9BCBFC1C4C7CACD59
:102EF000CFD2D5D8DBDEE1E4E7EAEDF0F4F7FAFD76
:102F0000808182838485868788898A8B8C8D8E8F49
:102F1000909192939495969798999A9B9C9D9E9F39
:102F2000A0A1A2A3A4A5A6A7A8A9AAABACADAEAF29
:102F3000B0B1B2B3B4B5B6B7B8B9BABBBCBDBEBF19
:102F4000C0C1C2C3C4C5C6C7C8C9CACBCCCDCECF09
:102F5000D0D1D2D3D4D5D6D7D8D9DADBDCDDDEDFF9
:102F6000E0E1E2E3E4E5E6E7E8E9EAEBECEDEEEFE9
:102F7000F0F1F2F3F4F5F6F7F8F9FAFBFCFDFEFFD9
:102F8000000102030405060708090A0B0C0D0E0FC9
:102F9000101112131415161718191A1B1C1D1E1FB9
:102FA000202122232425262728292A2B2C2D2E2FA9
:102FB000303132333435363738393A3B3C3D3E3F99
:102FC000404142434445464748494A4B4C4D4E4F89
:102FD000505152535455565758595A5B5C5D5E5F79
:102FE000606162636465666768696A6B6C6D6E6F69
:102FF000707172737475767778797A7B7C7D7E7F59
:1030000000020406080A0C0E10121416181A1C1ED0
:1030100020222426282A2C2E30323436383A3C3EC0
:1030200040424446484A4C4E50525456585A5C5EB0
:1030300060626466686A6C6E70727476787A7C7EA0
:103040007F7D7B79777573716F6D6B696765636180
:103050005F5D5B59575553514F4D4B494745434170
:103060003F3D3B39373533312F2D2B292725232160
:103070001F1D1B19171513110F0D0B090705030150
:10308000FFFDFBF9F7F5F3F1EFEDEBE9E7E5E3E140
:10309000DFDDDBD9D7D5D3D1CFCDCBC9C7C5C3C130
:1030A000BFBDBBB9B7B5B3B1AFADABA9A7A5A3A120
:1030B0009F9D9B99979593918F8D8B898785838110
:1030C00080828486888A8C8E90929496989A9C9E10
:1030D000A0A2A4A6A8AAACAEB0B2B4B6B8BABCBE00
:1030E000C0C2C4C6C8CACCCED0D2D4D6D8DADCDEF0
:1030F000E0E2E4E6E8EAECEEF0F2F4F6F8FAFCFEE0
:103100007F7F7F7F7F7F7F7F7F7F7F7F7F7F7F7FCF
:103110007F7F7F7F7F7F7F7F7F7F7F7F7F7F7F7FBF
:103120007F7F7F7F7F7F7F7F7F7F7F7F7F7F7F7FAF
:103130007F7F7F7F7F7F7F7F7F7F7F7F7F7F7F7F9F
:103400000309131E28313A40464C5054585B5E6104
:10341000636567696B6C6E6F7071727374757677C4
:10342000777879797A7A7B7B7C7C7C7D7D7D7E7EEA
:103430007E7E7F7F7F7F7F7F7F7F7F7F7F7F7F7F9E
:103440007F7F7F7F7F7F7F7F7F7F7F7F7F7E7E7E8F
:103450007E7D7D7D7C7C7C7B7B7A7A7979787777C1
:10346000767574737271706F6E6C6B69676563618A
:103470005E5B5854504C46403A31281E13090300F5
:10348000C6CCD5DBDFE3E5E7E9EAEBECEDEEEFEF09
:10349000F0F0F0F1F1F1F1F2F2F2F2F2F2F2F2F315
:1034A000F3F3F3F3F3F3F3F3F3F3F3F3F3F3F3F3EC
:1034B000F3F3F3F3F3F3F3F3F3F3F3F3F3F3F3F3DC
:1034C000F3F3F3F3F3F3F3F3F3F3F3F3F3F3F3F3CC
:1034D000F3F3F3F3F3F3F3F3F3F3F3F3F3F3F3F3BC
:1034E000F2F2F2F2F2F2F2F2F1F1F1F1F0F0F0EFC9
:1034F000EFEEEDECEBEAE9E7E5E3DFDBD5CCC60088
:1035000000283D42302D2C2B2C2D2E2F30323335E0
:1035100037393B3D3F414345484A4C4E5053555740
:10352000595B5D5F61636567696B6C6E7071737425
:10353000757778797A7B7C7D7D7E7E7F7F7F7F7FCC
:103540007F7F7F7F7F7F7E7E7D7D7C7B7A797877B2
:1035500075747371706E6C6B69676563615F5D5BD9
:1035600059575553504E4C4A484543413F3D3B39CE
:1035700037353332302F2E2D2C2B2C2D30423D2839
:1035800000E9E5FED4D7D7D7D6D4D2D0CECCCAC89E
:10359000C6C3C1BFBDBAB8B6B4B1AFADABA9A7A5DC
:1035A000A3A19F9E9C9A999795949391908F8D8CAF
:1035B0008B8A8988888786858584848483838383AE
:1035C0008383838383848484858586878888898AA6
:1035D0008B8C8D8F909193949597999A9C9E9FA197
:1035E000A3A5A7A9ABADAFB1B4B6B8BABDBFC1C3AF
:1035F000C6C8CACCCED0D2D4D6D7D7D7D4FEE5E968
:10360000F9F8F9F5EBE1DDDEE0E2E4E5E6E5E4E238
:10361000DED9D2CAC1B7ACA299918A868381808053
:103620008182838586888A8C8D8F909293959697D8
:1036300098999A9B9B9C9D9D9D9E9E9E9F9F9F9FC0
:103640009F9F9F9E9E9E9D9D9D9C9B9B9A999897B8
:1036500096959392908F8D8C8A88868583828180BF
:10366000808183868A9199A2ACB7C1CAD2D9DEE2A1
:10367000E4E5E6E5E4E2E0DEDDE1EBF5F9F8F900AA
:103680000708070B151F2322201E1C1B1A1B1C1EBC
:1036900022272E363F49545E676F767A7E7F7F7F82
:1036A0007F7E7D7B7A7876747371706E6D6B6A69DC
:1036B00068676665656464636362626261616161D3
:1036C00061616162626263636364656566676869BC
:1036D0006A6B6D6E7071737476787A7B7D7E7F7F96
:1036E0007F7F7E7A766F675E54493F362E27221E93
:1036F0001C1B1A1B1C1E2022231F150B070807006A
:103700001F313D444E5354565A5F64696E74767946
:103710007C7F7F7F7F7F7F7F7F7F7F7F7F7F7F7FBC
:103720007F7F7F7F7F7F7F7F7F7F7F7F7F7F7F7FA9
:103730007F7F7F7F7F7F7F7F7F7F7F7F7F7F7F7F99
:103740007F7F7F7F7F7F7F7F7F7F7F7F7F7F7F7F89
:103750007F7F7F7F7F7F7F7F7F7F7F7F7F7F7F7F79
:103760007F7F7F7F7F7F7F7F7F7F7F7F7F7F7F7F69
:103770007F7F7F7F7F7F7F7F7F7F7F7C7871684CBB
:103780002C1C120C0A0B0A05FDF3E9DFD4CAC0B7E2
:10379000AEA69E97918B8685828080808080808077
:1037A0008080808080808080808080808080808019
:1037B0008080808080808080808080808080808009
:1037C00080808080808080808080808080808080F9
:1037D00080808080808080808080808080808080E9
:1037E00080808080808080808080808080808080D9
:1037F000808080808087919DACC4CBD4DDF2FAFAC2
:1038000022002400260028002B002D003000330069
:10381000360039003D004000440048004C00510093
:1038200056005B00600066006C0073007900810048
:10383000880090009900A200AC00B600C100CC0046
:10384000D800E500F300010110012101320144011B
:1038500057016C0181019801B001CA01E501020222
:103860002102410264028802AE02D7020303300340
:1038700061039403CB03050442048304C7041005C9
:103880005D05AF0505066106C2062907960709080A
:10389000830805098E09200ABA0A5D0B0A0CC10CBF
:1038A000840D510E2B0F121007110A121D13401414
:1038B0007415BA1614188319071BA31C571E24204D
:1038C0000E22142439267F28E82A752D2930063344
:1038D0000F364539AD3C49401B442848734CFE50D7
:1038E000CF55EA5A51600C661D6C8B725A799280E2
:1038F00037885090E598FDA19FABD3B5A3C00000D9
:10390000EF92FF920F931F937B018C0120E030E038
:1039100040E05FE40E94501F88238CF020E030E0FC
:1039200040E05FE4C801B7010E94F81D0E94DE1F5D
:103930009B01AC01205030404040504806C0C801B7
:10394000B7010E94DE1F9B01AC01B901CA011F91A2
:103950000F91FF90EF900895A0E0B0E0E2EBFCE162
:103960000C941C2CDC012B01FA019C91923008F480
:1039700039C1EB018881823008F433C1943069F495
:10398000843009F02FC111969C9111978981981765
:1039900009F428C1ACE2B1E025C1843009F421C1A9
:1039A0008230A9F4923009F01DC19A01AD0188E07E
:1039B000EA010990AE01E90109929E018150C1F727
:1039C000E201898111969C918923818308C19230FB
:1039D00009F407C112962D903C901397EB018A8150
:1039E0009B811496AD90BD90CD90DC901797EC80A4
:1039F000FD800E811F819101281B390BB90137FF12
:103A000004C066277727621B730B603271050CF0C8
:103A100061C0121613066CF537014801062E04C06A
:103A200096948794779467940A94D2F721E030E0D3
:103A300040E050E004C0220F331F441F551F6A9519
:103A4000D2F721503040404050402E213F214023AA
:103A50005123211531054105510521F021E030E0C8
:103A600040E050E079018A01E628F7280829192961
:103A70003CC0232BD1F1260E371E35014601062E00
:103A800004C096948794779467940A94D2F721E0BF
:103A900030E040E050E004C0220F331F441F551FA8
:103AA0006A95D2F721503040404050402A213B21B6
:103AB0004C215D21211531054105510521F021E001
:103AC00030E040E050E059016A01A628B728C82834
:103AD000D9280BC0821593052CF01C01AA24BB2405
:103AE000650103C0EE24FF24870111969C91D20149
:103AF00011968C91981709F445C0992339F0A801C3
:103B000097012A193B094C095D0906C0A6019501D8
:103B10002E193F09400B510B57FD08C0118233820B
:103B2000228224833583468357831DC081E08183AD
:103B30003382228288279927DC01821B930BA40BF6
:103B4000B50B84839583A683B7830DC0220F331FE3
:103B5000441F551F24833583468357838281938175
:103B60000197938382832481358146815781DA01CD
:103B7000C9010197A109B1098F5F9F4FAF4FBF43A3
:103B800028F30BC0918333822282EA0CFB1C0C1DAC
:103B90001D1DE482F5820683178383E080832481E0
:103BA00035814681578157FF1AC0C901AA2797FD61
:103BB000A095BA2F81709070A070B07056954795FF
:103BC00037952795822B932BA42BB52B8483958334
:103BD000A683B78382819381019693838283DF01D9
:103BE00001C0D201CD01CDB7DEB7E2E10C94382C93
:103BF000A0E2B0E0EEEFFDE10C94282C69837A831B
:103C00008B839C832D833E834F835887E9E0EE2E80
:103C1000F12CEC0EFD1EB701CE0101960E9456213B
:103C20008E010F5E1F4FB801CE0105960E945621EE
:103C30008A8991E089278A8BAE01475E5F4FB80180
:103C4000C7010E94AC1C0E948120A096E6E00C9463
:103C5000442CA0E2B0E0EFE2FEE10C94282C698352
:103C60007A838B839C832D833E834F835887F9E02F
:103C7000EF2EF12CEC0EFD1EB701CE0101960E9435
:103C800056218E010F5E1F4FB801CE0105960E948E
:103C90005621AE01475E5F4FB801C7010E94AC1CC0
:103CA0000E948120A096E6E00C94442CA0E2B0E0B3
:103CB000ECE5FEE10C941C2C69837A838B839C8356
:103CC0002D833E834F835887BE01675F7F4FCE01B0
:103CD00001960E945621BE016F5E7F4FCE01059670
:103CE0000E9456219985923088F089898230C8F0E7
:103CF000943019F4823051F404C0843029F49230A5
:103D000081F48CE291E0C6C0923049F420E09A85BB
:103D10008A89981321E02A87CE010996BBC0823098
:103D200049F420E09A858A89981321E02A8BCE01F4
:103D30004196B0C02D843E844F8458886D887E881B
:103D40008F88988CEE24FF248701AA24BB24650168
:103D500040E050E060E070E0E0E0F0E0C101817040
:103D60009070892BE9F0E60CF71C081D191D9A01CB
:103D7000AB012A0D3B1D4C1D5D1D80E090E0A0E0D5
:103D8000B0E0E614F7040805190520F481E090E09E
:103D9000A0E0B0E0BA01A901480F591F6A1F7B1FBC
:103DA000AA0CBB1CCC1CDD1C97FE08C081E090E077
:103DB000A0E0B0E0A82AB92ACA2ADB2A3196E0326C
:103DC000F10549F0660C771C881C991C56944794A1
:103DD00037942794C3CFFA85EA892B893C898B8550
:103DE0009C85280F391F2E5F3F4F17C0CA01817075
:103DF0009070892B61F016950795F794E79480E011
:103E000090E0A0E0B0E8E82AF92A0A2B1B2B76956F
:103E10006795579547952F5F3F4F77FDE7CF0CC0CC
:103E2000440F551F661F771F17FD4160EE0CFF1CE6
:103E3000001F111F21503040403090E0590790E0A2
:103E4000690790E4790760F32B8F3C8FDB01CA018F
:103E50008F779070A070B07080349105A105B10586
:103E600061F447FD0AC0E114F1040105110529F0D0
:103E7000405C5F4F6F4F7F4F40781A8EFE1711F0F6
:103E800081E08A8F4D8F5E8F6F8F78A383E0898F5B
:103E9000CE0149960E948120A096E2E10C94382C34
:103EA000A8E1B0E0E6E5FFE10C94282C69837A8371
:103EB0008B839C832D833E834F83588789E0E82E34
:103EC000F12CEC0EFD1EB701CE0101960E94562189
:103ED0008E010F5E1F4FB801CE0105960E9456213C
:103EE0008985823040F08989823028F0B801C70185
:103EF0000E94CE2101C08FEF6896E6E00C94442C1E
:103F0000A8E0B0E0E6E8FFE10C94252C9B01AC01B1
:103F100083E08983DA01C9018827B7FD8395992752
:103F2000AA27BB27B82E211531054105510519F4E3
:103F300082E089833AC08823A9F0203080E03807E6
:103F400080E0480780E8580729F460E070E080E0EE
:103F50009FEC30C0EE24FF248701E21AF30A040B21
:103F6000150B02C079018A018EE1C82ED12CDC82AA
:103F7000CB82ED82FE820F831887C801B7010E94B1
:103F8000322001971816190684F4082E04C0EE0C8E
:103F9000FF1C001F111F0A94D2F7ED82FE820F83CF
:103FA0001887C81AD90ADC82CB82BA82CE01019660
:103FB0000E9481202896E9E00C94412CACE0B0E00E
:103FC000E4EEFFE10C942C2C69837A838B839C8331
:103FD000BE016B5F7F4FCE0101960E9456218D81FD
:103FE000823061F1823050F1843021F48E81882357
:103FF00051F12EC02F81388537FD20C06E812F31C1
:1040000031051CF06623F9F023C08EE190E0821B9D
:10401000930B29853A854B855C8504C05695479559
:10402000379527958A95D2F76623B1F0509540953C
:10403000309521953F4F4F4F5F4F0EC020E030E04D
:1040400040E050E009C02FEF3FEF4FEF5FE704C0C3
:1040500020E030E040E050E8B901CA012C96E2E0EF
:104060000C94482CEF92FF920F931F937B018C01CD
:1040700080E0E81680E0F80681E0080780E0180795
:1040800088F48FEFE816F1040105110531F028F0EE
:1040900088E090E0A0E0B0E017C080E090E0A0E011
:1040A000B0E012C080E0E81680E0F80680E0080783
:1040B00081E0180728F088E190E0A0E0B0E004C0BB
:1040C00080E190E0A0E0B0E020E230E040E050E0AD
:1040D000281B390B4A0B5B0B04C016950795F79408
:1040E000E7948A95D2F7F701EC5CFE4F8081281B9C
:1040F000310941095109C9011F910F91FF90EF90BA
:104100000895DF92EF92FF920F931F93FC01E480DA
:10411000F58006811781D1808081823048F480E06B
:1041200090E0A0E1B0E0E82AF92A0A2B1B2BA5C0F9
:10413000843009F49FC0823021F4EE24FF248701EB
:1041400005C0E114F1040105110519F4E0E0F0E007
:1041500096C0628173819FEF623879070CF05BC073
:1041600022E83FEF261B370B2A3131052CF020E0E7
:1041700030E040E050E02AC0B801A701022E04C0A0
:1041800076956795579547950A94D2F781E090E028
:10419000A0E0B0E004C0880F991FAA1FBB1F2A959A
:1041A000D2F70197A109B1098E219F21A023B12344
:1041B0000097A105B10521F081E090E0A0E0B0E01A
:1041C0009A01AB01282B392B4A2B5B2BDA01C90151
:1041D0008F779070A070B07080349105A105B10503
:1041E00039F427FF09C0205C3F4F4F4F5F4F04C099
:1041F000215C3F4F4F4F5F4FE0E0F0E02030A0E008
:104200003A07A0E04A07A0E45A0710F0E1E0F0E026
:1042100079018A0127C06038710564F5FB01E15816
:10422000FF4FD801C7018F779070A070B0708034B5
:104230009105A105B10539F4E7FE0DC080E490E0D9
:10424000A0E0B0E004C08FE390E0A0E0B0E0E80EB2
:10425000F91E0A1F1B1F17FF05C016950795F79437
:10426000E794319687E016950795F794E7948A9539
:10427000D1F705C0EE24FF248701EFEFF0E06E2FA9
:10428000679566276795902F9F77D794DD24D794FD
:104290008E2F8695492F462B582F5D29B701CA01CD
:1042A0001F910F91FF90EF90DF900895FC01DB01CB
:1042B000408151812281622F6F7770E0221F222777
:1042C000221F9381892F880F822B282F30E0991F7E
:1042D0009927991F11969C93119721153105A9F5DE
:1042E000411551056105710511F482E037C082E87E
:1042F0009FEF13969C938E9312979A01AB0167E000
:10430000220F331F441F551F6A95D1F783E08C930A
:104310000DC0220F331F441F551F12968D919C9183
:104320001397019713969C938E931297203080E0F9
:10433000380780E0480780E4580758F314962D9317
:104340003D934D935C93179708952F3F310579F472
:10435000411551056105710519F484E08C930895A8
:1043600064FF03C081E08C9312C01C9210C02F57D1
:10437000304013963C932E93129783E08C9387E002
:10438000440F551F661F771F8A95D1F770641496E6
:104390004D935D936D937C93179708951F93DC0164
:1043A000FB019C91923008F447C08081823008F470
:1043B00043C0943051F411961C91843099F5818159
:1043C000682F70E0611B71093FC0843021F092308A
:1043D00031F48230B9F18181882389F12DC01196A1
:1043E0001C9111978230F1F081811817D9F412963F
:1043F0002D913C911397828193818217930794F0BA
:1044000028173907BCF014968D919D910D90BC91A1
:10441000A02D2481358146815781281739074A0705
:104420005B0718F4112341F00AC082179307A40711
:10443000B50740F4112319F061E070E005C06FEF9B
:104440007FEF02C060E070E0CB011F910895FF9202
:104450000F931F93CF93DF93129A8091A80E882316
:1044600029F081E090E00E942B1502C0C895C89504
:104470001298FF2400E010E0C0E0D0E01695079508
:10448000D695C79513988091A80E882329F085E0CA
:1044900090E00E942B1502C0C895C895009B10683B
:1044A000019BD068139A8091A80E882329F085E09B
:1044B00090E00E942B1502C0C895C895F39480E146
:1044C000F816E1F610933D0C00933C0CD093410C90
:1044D000C093400CDF91CF911F910F91FF900895F1
:1044E000FF920F931F93CF93DF930E942722809117
:1044F0003C0C90913D0C97FD06C08091400C909132
:10450000410C97FF27C081E090E00E942B1500E04E
:1045100010E0C0E0D0E0FF24000F111FCC0FDD1F22
:104520001398C895C895C895C895009B0160019BD4
:10453000C160139A88E090E00E942B15F39480E10B
:10454000F81651F710933F0C00933E0CD093430C98
:10455000C093420CDF91CF911F910F91FF9008956E
:104560000F931F9380EB98E00E946E2380E00E94DF
:104570001C1480E790E00E9424140E94C21389E179
:1045800090E00E94502800E040E758E0602F8DE066
:104590000E94B62781E090E00E9450281DE040E094
:1045A00050E0602F812F0E94FE131F5F1231B9F778
:1045B0000F5F0D3049F780EB98E00E946E2341E0D9
:1045C0006FEF80E00E94D92640E758E06CE08DE074
:1045D0000E94B62742E958E06FE08DE00E94B627BE
:1045E00083E090E00E94502841E858E06CE08DE0C4
:1045F0000E94B62782E090E00E94502840E758E0F1
:104600006CE08DE00E94B62788E290E00E9450287E
:104610008AE090E00E9450280E94C21384E190E05A
:104620000E9450281F910F91089590E026E130E0FC
:10463000829FF001839FF00D929FF00D1124E555AC
:10464000F14F628708956093910E089590E026E1FE
:1046500030E0829FF001839FF00D929FF00D1124B6
:10466000E555F14F13861182089590E026E130E080
:10467000829FF001839FF00D929FF00D1124E5556C
:10468000F14F81E0838B089590E026E130E0829F36
:10469000F001839FF00D929FF00D1124E555F14F2D
:1046A0006187089590E026E130E0829FF001839FCA
:1046B000F00D929FF00D1124E555F14F648308959C
:1046C00090E026E130E0829FF001839FF00D929F01
:1046D000F00D1124E555F14F658308959093060F71
:1046E0008093050F8FE680930B0F1092600CEBEA1E
:1046F000FEE021E08FEF98E1208310868683878398
:1047000014861182958376963FE0E330F307A1F794
:104710000895DC01ED91FC911197AF014F5F5F4F60
:1047200011965C934E93E4912E2F30E0E7FF13C077
:104730002F7730703695322F222737952795FA013B
:104740004F5F5F4FE4918E2F8F77280F311DE7FD6C
:10475000F1CF4D935C93C90108950E949F15089570
:10476000EF92FF920F931F93CF93DF93182F062F93
:10477000F42EE22EC82FD0E086E190E0C89FF00131
:10478000C99FF00DD89FF00D1124E555F14F838599
:10479000882321F08181882309F0ACC0EE2091F4B8
:1047A00086E190E0C89FF001C99FF00DD89FF00D01
:1047B0001124E555F14F138A8285882309F09AC0A8
:1047C000108698C0133059F481E091E09093930ED5
:1047D0008093920E81E08093910E0F2D08C060E0CF
:1047E000812F0E949F156F2D812F0E9480150F37FA
:1047F00099F486E190E0C89FF001C99FF00DD89F21
:10480000F00D1124E555F14F8091080F878789E05D
:104810009FE0958B848B30C089E0089FC0011124F4
:10482000E091050FF091060FE80FF91F33964591BF
:1048300054914115510571F486E190E0C89FF00153
:10484000C99FF00DD89FF00D1124E555F14F158A41
:10485000148A12C0FA01249186E190E0C89FF00109
:10486000C99FF00DD89FF00D1124E555F14F278712
:104870004F5F5F4F558B448B86E190E0C89FD0011E
:10488000C99FB00DD89FB00D1124A555B14F5096BA
:104890001C9250971A961C921A971C960C931C9770
:1048A00011961C9211972FEF19962C931997189621
:1048B000EC9218978BE090E0C89FF001C99FF00D33
:1048C000D89FF00D1124EE0FFF1FE355F14FF0823A
:1048D00051961C92519781E01B968C931B9753968F
:1048E0001C92539752961C92529714961C921497AE
:1048F00016962C93DF91CF911F910F91FF90EF901F
:104900000895CF92DF92FF920F931F93CF93DF937F
:10491000E4EBFEE08181282F332727FD309580814D
:10492000280F311D2F3F310519F014F02FEF30E023
:10493000C90137FF02C080E090E0808376964FE0A7
:10494000EC30F40739F78091600C882309F027C117
:1049500043C1E0910E0FF0910F0F9F012F5F3F4F6A
:1049600030930F0F20930E0F44914F3F69F5A9012B
:104970004F5F5F4F50930F0F40930E0FF9018491DB
:104980008F3219F41092600C18C1863009F0FAC009
:10499000FA013196CF01019690930F0F80930E0F7D
:1049A000E491E33529F49093120F8093110FEAC03C
:1049B000E53409F0E7C08091110F9091120F9093A8
:1049C0000F0F80930E0FDEC047FF02C04093070F0A
:1049D000542F5F70842F90E0807F9070803B910512
:1049E00029F1803C910579F18039910509F042C0A7
:1049F000C9010196F9014491019690930F0F80939C
:104A00000E0F0197FC012491852F90E08C9FF001FF
:104A10008D9FF00D9C9FF00D1124E555F14F808185
:104A2000882309F4AFC0220F648552C0C9010196E2
:104A3000F9014491019690930F0F80930E0F019707
:104A4000FC01249153C02F5F3F4F30930F0F2093F1
:104A50000E0F21503040F9012491852F90E08C9F5A
:104A6000F0018D9FF00D9C9FF00D1124E555F14F45
:104A7000248788C08091070F582F5F7090E0807F57
:104A80009070803B910541F1803C910509F46EC026
:104A90008039910509F076C02F5F3F4F30930F0F9B
:104AA00020930E0F21503040F9012491852F90E082
:104AB0008C9FD0018D9FB00D9C9FB00D1124A555EA
:104AC000B14F8C91882309F45DC0220F1C966C9124
:104AD000852F0E94B02356C02F5F3F4F30930F0F9A
:104AE00020930E0F21503040F9012491473071F48A
:104AF000852F90E08C9FF0018D9FF00D9C9FF00D15
:104B00001124E555F14F220F27833CC04B3071F43F
:104B1000852F90E08C9FF0018D9FF00D9C9FF00DF4
:104B20001124E555F14F220F26832CC04C3571F42A
:104B3000852F90E08C9FF0018D9FF00D9C9FF00DD4
:104B40001124E555F14F220F24831CC04436D1F4C3
:104B5000852F90E08C9FF0018D9FF00D9C9FF00DB4
:104B60001124E555F14F220F25830CC0852F90E0CD
:104B70008C9FF0018D9FF00D9C9FF00D1124E55549
:104B8000F14F44878EE09FE00E94892390930D0FA0
:104B900080930C0F1092040F1092030F02C0C6E115
:104BA000D0E06091030F7091040F80910C0F9091F1
:104BB0000D0F6817790709F4CCCE6F5F7F4F7093A4
:104BC000040F6093030F8091090F90910A0F0196D3
:104BD00090930A0F8093090F02E71EE0CCEADEE013
:104BE000FF24BFEFCB2ED12C8A89882309F05EC029
:104BF0008B899C89892B09F456C09F858E859817CF
:104C000008F04CC050C08B852B893C898F37E9F464
:104C1000D9018D91BC8BAB8B8F3F01F1F901618183
:104C20001196BC8BAB8BE82FF0E0EE0FFF1FE75423
:104C3000F74F0190F081E02D8F2D0995EB89FC89CC
:104C400081918E87FC8BEB8B28C0A9014F5F5F4F52
:104C50005C8B4B8BF90184918F3F21F418821C8A65
:104C60001B8A21C04F5F5F4F5C8B4B8B4150504084
:104C7000FA01649190E0880F991F8754974FFC01C7
:104C8000259134918F2DF9010995EB89FC89319695
:104C9000FC8BEB8B3197E491EE871F869F858E8589
:104CA000981709F4B0CF8F858F5F8F878A85882307
:104CB00019F420E030E06BC088898F3F11F08F5FDE
:104CC000888B9F81992309F45CC02885222309F4ED
:104CD00058C08E81882309F454C040910B0F44239F
:104CE00009F44FC0899FC001112480509F4F892F24
:104CF000992730E0B901869F9001879F300D969FDC
:104D0000300D112420503F4F232F33278D8190E009
:104D1000FC012E9FC0012F9F900D3E9F900D1124EE
:104D200080509F4F892F9927242F30E0AC01429F5C
:104D3000C001439F900D529F900D112480509F4FB2
:104D4000292F33278B818823F1F0EA81F0E0E050AE
:104D5000F24DE491E058E89FC001112480509F4F2C
:104D6000892F9927B601681B790B629FC001639F49
:104D7000900D729F900D112480509F4F292F332743
:104D800002C020E030E08A819C81890F8A83F8018B
:104D90002083F394065F1F4F6696F4E0FF1609F038
:104DA00023CFDF91CF911F910F91FF90DF90CF9094
:104DB00008951F93CF93DF93582F89E0589FC00128
:104DC00011242091050F3091060F280F391FC901BA
:104DD0000396FC01A591B491F90184918150823030
:104DE00010F413E01DC08091C20E8823B1F08091B1
:104DF000CE0E851711F4442381F48091D80E8823B8
:104E000071F08091E40E851711F4442341F49091E0
:104E1000D20E8091E80E891710F411E001C012E063
:104E2000212F30E0FD01449186E190E0289FE001D0
:104E3000299FD00D389FD00D1124C555D14F4F87D4
:104E40001196BD8BAC8B188A8BE090E0289FF00107
:104E5000299FF00D389FF00D1124EE0FFF1FE35531
:104E6000F14F80E5808368878FEF89871A861B8AD8
:104E7000198A21E02B871A8A5D8729831C828E83F9
:104E8000133049F481E091E09093930E8093920E59
:104E90002093910E08C060E5812F0E9480156A89D9
:104EA000812F0E949F15DF91CF911F910895FF924E
:104EB0000F931F93082FF62E0E94801510E08BE0B1
:104EC00090E0089FF001099FF00D189FF00D11244C
:104ED000EE0FFF1FE355F14FF0821F910F91FF90EE
:104EE0000895962F482F50E02BE030E0429FF001CC
:104EF000439FF00D529FF00D1124EE0FFF1FE3555D
:104F0000F14F6081691B60830E9480150895482FCE
:104F100050E02BE030E0429FF001439FF00D529FA4
:104F2000F00D1124EE0FFF1FE355F14F9081690F33
:104F300060830E948015089530913D0F20E010C0DD
:104F4000822F90E0FC01EE0FFF1FE80FF91FEA51DE
:104F5000F44FA081B181A05CBD4F82818C932F5F03
:104F6000231770F308958093000108951F93CF9342
:104F7000DF93FA01749131961491C72FD0E0AF01FD
:104F80004F5F5F4F9EE1699F90011124280F311DF3
:104F900060E00CC08491875E8D939F5F3196971778
:104FA000C8F36F5F4C0F5D1F225E3F4F611730F4F7
:104FB000D901A05CBD4FFA0190E0F1CFDF91CF9114
:104FC0001F9108951F93CF93DF93A82FFB01749136
:104FD0003196B491C72FD0E0AF014F5F5F4F60E0D3
:104FE00016C0F9018491E12FF0E0EE0FFF1FEE0FE4
:104FF000FF1FEB5EF04F80839F5F2F5F3F4F192FA6
:105000001A0F971770F3A70F6F5F4C0F5D1F6B1789
:1050100018F49A0190E0F3CFDF91CF911F9108959A
:105020000F9350E012C0F0E0EE0FFF1FEE0FFF1FD6
:10503000ED5EF04F308341839F5F385FE92FE80FCB
:10504000921788F3820F5F5F485F501718F4362F6E
:1050500090E0F4CF0F91089580913E0F8823F9F0EE
:1050600080913F0F8823C1F480913B0F80933F0FC5
:105070009091400FE92FF0E0E050FF4F808187B919
:1050800080913C0F890F8093400F882311F08D3061
:1050900031F410923E0F0895815080933F0F089590
:1050A0000F931F93CF93DF938C01C0E0D0E007C034
:1050B0000E9429148823E1F30E942C142196C01722
:1050C000D107B4F3DF91CF911F910F9108957F9293
:1050D0008F929F92AF92BF92CF92DF92EF92FF9208
:1050E0000F931F93CF93DF93782E862EEA01FA0158
:1050F000C590D490FA013296A590B49000E016C005
:10510000FC01EE0DFF1D3296EE0FFF1FEC0FFD1F91
:1051100045915491692D812F870D0E94FE131F5FC9
:10512000812F90E08C159D055CF30F5F802F90E040
:105130008A159B055CF48C9D70018D9DF00C9C9DE7
:10514000F00C112410E0902E980CEACFDF91CF9153
:105150001F910F91FF90EF90DF90CF90BF90AF9095
:105160009F908F907F9008952F923F924F925F92E1
:105170006F927F928F929F92AF92BF92CF92DF9267
:10518000EF92FF920F931F93DF93CF9300D00F9274
:10519000CDB7DEB710923D0F80910001882309F44E
:1051A0009AC063E1862E6FE0962E7724F4019181F8
:1051B000903E08F071C08081382F3695369536952F
:1051C000282F277019F0F2E0F98302C081E089836B
:1051D000892F869586958695977019F052E0652EF1
:1051E00002C066246394B92EAA241501220E311C34
:1051F0009EE1899F80011124030F111DCC24DD2421
:1052000040C02A813B81200F311FF7017081793125
:10521000E8F060913D0F693110F5862F90E0FC01B8
:10522000EE0FFF1FE80FF91FEA51F44F318320837F
:105230007283872F0E943E1470913D0FF701708397
:105240007F5F70933D0F7150793148F44A815B81E3
:10525000440D551D9101672F872D0E94CF148A811F
:105260009B8101969B838A830894E11CF11C9981A0
:10527000891738F20894C11CD11C025E1F4FC61456
:1052800058F45C2C442480E4E82E82E0F82EE00EF2
:10529000F11E1B821A82B5CF7394E4E0F0E08E0E0B
:1052A0009F1EFAE07F1609F081CF30913D0F20E07C
:1052B00010C0822F90E0FC01EE0FFF1FE80FF91FD6
:1052C000EA51F44FA081B181A05CBD4F82818C93E3
:1052D0002F5F231770F30F900F900F90CF91DF91F6
:1052E0001F910F91FF90EF90DF90CF90BF90AF9004
:1052F0009F908F907F906F905F904F903F902F90F6
:1053000008958F929F92AF92BF92CF92DF92EF92C9
:10531000FF920F931F9380919C0E882381F080E071
:1053200090E0A0ECBFEB80939E0E90939F0EA09315
:10533000A00EB093A10E10929C0E10920F0120911E
:105340009E0E30919F0E4091A00E5091A10E609143
:1053500014017091150180911601909117010E941E
:10536000291E7B018C0160931401709315018093B9
:105370001601909317012091A20E3091A30E409137
:10538000A40E5091A50E60911001709111018091B1
:105390001201909113010E94291E5B016C01609320
:1053A000100170931101809312019093130180906A
:1053B0000D0190900E01C801B7010E94801C7B0175
:1053C0008C01F4016083C601B5010E94801C862F08
:1053D000F4016183EA94F4EEFE1508F047C041E061
:1053E0006FEF82E00E94D92681E080930F0180E078
:1053F00090E0A8EEB2E48093140190931501A0937D
:105400001601B093170180E090E0A8EDB2E480931C
:10541000100190931101A0931201B093130180E049
:1054200090E0A0E0B0E080939E0E90939F0EA0933A
:10543000A00EB093A10E8093A20E9093A30EA09302
:10544000A40EB093A50EE0910D01F0910E018081A4
:10545000882331F480919B0E8F5F80939B0E1FC039
:1054600080919A0E8F5F80939A0E19C089508A3C62
:10547000B0F041E06FEF81E00E94D9268091A20E4A
:105480009091A30EA091A40EB091A50EB058809358
:10549000A20E9093A30EA093A40EB093A50E1F91FD
:1054A0000F91FF90EF90DF90CF90BF90AF909F90C3
:1054B0008F9008950F9304E021E04091420F6AE03D
:1054C00081E00E94102821E04091440F6EED86E0BB
:1054D0000E941028E0910D01F0910E018081482F6B
:1054E00050E08091410F282F30E0C90105968417C4
:1054F0009507BCF5295F3F4F2417350794F181814B
:10550000682F70E08091420F282F30E0CB01079682
:105510008217930734F1215E3F4F261737070CF1AE
:1055200041E06FEF80E00E94D92680919E0E90911D
:105530009F0EA091A00EB091A10EB05880939E0E28
:1055400090939F0EA093A00EB093A10EE0910D0139
:10555000F0910E01618170E06C5070402091420F1B
:1055600041C08091430F282F30E0CA01079682176F
:1055700093070CF44DC04B5F5F4F421753070CF07D
:1055800047C08181482F50E08091440F282F30E0A0
:10559000CA01079682179307DCF1215E3F4F24175B
:1055A0003507B4F141E06FEF80E00E94D926809189
:1055B0009E0E90919F0EA091A00EB091A10EB0589A
:1055C00080939E0E90939F0EA093A00EB093A10E79
:1055D000E0910D01F0910E01618170E06C5070401E
:1055E0002091440F621B7109882777FD8095982FC1
:1055F0000E94801F2FE135E84BEE5DE30E94561EAE
:105600006093A20E7093A30E8093A40E9093A50EA8
:1056100081E090E00E9450280F9108950F931F930E
:10562000DF93CF93CDB7DEB764970FB6F894DEBFA4
:105630000FBECDBFDE011196E8E1F1E084E10190FB
:105640000D928150E1F7E0919A0EEA3008F58091D1
:105650009B0E8A30E8F4F0E0EE0FFF1F8E010F5F23
:105660001F4FE00FF11F4081518162E08AE00E94EC
:10567000672880919B0E90E0880F991F080F191FD3
:10568000F8014081518162E080E10E9467281CC0DE
:1056900080E00E94B32780E090E0A0E0B0E080933B
:1056A0009E0E90939F0EA093A00EB093A10E809398
:1056B000A20E9093A30EA093A40EB093A50E81E02A
:1056C00080930F0180939D0E64960FB6F894DEBF11
:1056D0000FBECDBFCF91DF911F910F9108951F9302
:1056E00080E00E941315182F81E00E94131514FF0B
:1056F0000AC09091420F993030F010FF02C09350D1
:105700000DC092500BC015FF0BC09091420F983BFB
:1057100038F410FF02C09D5F01C09E5F9093420F5E
:1057200084FF0AC09091440F993030F010FF02C0FE
:1057300093500DC092500BC085FF0BC09091440F49
:10574000983B38F480FF02C09D5F01C09E5F90933C
:10575000440F13FF0CC080910F01882341F080910A
:105760009D0E882321F481E080939C0E23C012FFBC
:1057700021C080910F018823E9F081E00E94B327C6
:1057800010929A0E10929B0E80E090E0A0E0B0E0A4
:1057900080939E0E90939F0EA093A00EB093A10EA7
:1057A0008093A20E9093A30EA093A40EB093A50E87
:1057B00010929D0E1F91089588E892E20E946E2338
:1057C0008FEC98E00E94241485E00E941C148FEC5A
:1057D00098E00E941F144FE05AE160E080E00E94D0
:1057E0006728E0910D01F0910E01128263EA70E2E8
:1057F00081E00E94E22763EA70E286E00E94E227ED
:10580000E0910D01F0910E0184E780838CE68183A5
:105810008AE08093410F8EED8093430F85E580935E
:10582000420F8093440F0E940E2B0E946F2B0E9408
:105830005A2A0E948129F7CF2F923F924F925F926E
:105840006F927F928F929F92AF92BF92CF92DF9290
:10585000EF92FF920F931F93CF93DF93CDB7DEB7F5
:10586000CA1BDB0B0FB6F894DEBF0FBECDBF099489
:105870002A88398848885F846E847D848C849B84E0
:10588000AA84B984C884DF80EE80FD800C811B81EE
:10589000AA81B981CE0FD11D0FB6F894DEBF0FBE1D
:0A58A000CDBFED010895F894FFCF8D
:1058AA000100408891D2E4ADB5B6BEBFFF130F0127
:1058BA000000D8420000E842A920D52001212D216C
:1058CA0059218521B121DD2109223522000000005C
:1058DA00000000000001020203030303040404049D
:1058EA000404040405050505050505050505050562
:1058FA000505050506060606060606060606060642
:10590A00060606060606060606060606060606062D
:10591A000606060607070707070707070707070711
:10592A0007070707070707070707070707070707FD
:10593A0007070707070707070707070707070707ED
:10594A0007070707070707070707070707070707DD
:10595A0007070707080808080808080808080808C1
:10596A0008080808080808080808080808080808AD
:10597A00080808080808080808080808080808089D
:10598A00080808080808080808080808080808088D
:10599A00080808080808080808080808080808087D
:1059AA00080808080808080808080808080808086D
:1059BA00080808080808080808080808080808085D
:1059CA00080808080808080808080808080808084D
:0459DA0008080808A9
:00000001FF
